:1000000000308A00E7280000831A0A28A500030EA2
:10001000A6000F288312A500030EA600A6140A0846
:10002000AD008A018313A50E0408A7002008A800CC
:100030002108A9002208AA002308AB002408AC006C
:1000400083128C308400001C27280C188C28270869
:1000500084002808A0002908A1002A08A2002B0873
:10006000A3002C08A4002D088A00260E830083120A
:10007000250EA618831609002030C600C201C30150
:10008000C401C5013D08A3003C08A2003B08A10033
:100090003A08A0000310201C5B283E08C2073F0856
:1000A00003183F0FC30740080318400FC407410857
:1000B0000318410FC507C50CC40CC30CC20CA30C1C
:1000C000A20CA10CA00CC60B4A289D28A101A201DC
:1000D000A001A3014008031D70283F0803198A28C6
:1000E0001030C1000310BD0DBE0DA00DA30D4008C2
:1000F0002302031D7D283F082002031C86283F0899
:10010000A002031CA3034008A3020314A10DA20D27
:10011000C10B72280000C5283208BD003108BC00A0
:100120003008BB002F08BA004130C100C630C00003
:100130004E30BF006D30BE003C2839302007AF0084
:100140002108B000303003183130B0072208B10068
:10015000003003180130B1072308B2000030031843
:100160000130B2073108A0003208A100A201A301AA
:100170003208BC003108BB003208BE003108BD00A7
:100180007F30C000FF30BF0066282008A100230890
:10019000A20022088F0021088E003314B60A03192A
:1001A000B70A0C108A112728393084000008031977
:1001B000E6280230A100A001A00BDC28A10BDB285F
:1001C0009730A000A00BE228800BD92800348401CE
:1001D0001F308305713083168F0083121F1383161F
:1001E0001F109F101F119F11073083129900AE013D
:1001F0000130AF00B001B101B2013310B601B70157
:100200001F1383161F149F101F119F111F169F1677
:100210001F1383129F171F1483160108C73908384C
:1002200081008530831290000030A10006389200D2
:10023000FF30831692000515831295019501073052
:1002400099008316050806308312A000A00B26290A
:10025000000019088C11831699010C14C030831208
:100260008B04713083168F0083123608643C031DA3
:100270006329B708031D632905158316051164302A
:100280008312B900D420051183160511783083122A
:10029000B900D4200515831605115A308312B90010
:1002A000D4200511831605110A308312B900D42019
:1002B00005158316051164308312B900D420051189
:1002C0008316051183123608B03C031DB229370886
:1002D000043C031DB22905158316051164308312F1
:1002E000B900D42005118316051178308312B900A6
:1002F000D4200515831605115A308312B900D42075
:100300000511831605110A308312B900D420051592
:100310008316051164308312B900D42005118316A9
:100320000511831205158316051164308312B90077
:10033000D42005118316051178308312B900D4201A
:100340000515831605115A308312B900D4200515FE
:100350008316051164308312B900D4200511831669
:10036000051183123608D03C031DD7293708073CF6
:10037000031DD729051583160511C8308312B9004E
:10038000D42005118316051178308312B900D420CA
:1003900005158316051102308312B800C830B90064
:1003A000D420B80BCE290511831605118312360807
:1003B000B83C031D3F2A37080B3C031D3F2A051597
:1003C0008316051164308312B900D42005118316F9
:1003D000051178308312B900D42005158316051154
:1003E0005A308312B900D420051583160511C83080
:1003F0008312B900D42005118316051178308312B9
:10040000B900D42005158316051102308312B800F7
:10041000C830B900D420B80B082A0511831605117D
:100420000A308312B900D4200515831605116430F3
:100430008312B900D4200511831605118312051506
:100440008316051164308312B900D4200511831678
:10045000051178308312B900D420051583160511D3
:100460005A308312B900D420051583160511643063
:100470008312B900D42005118316051183123608A2
:10048000683C031D872A3708103C031D872A051581
:100490008316051164308312B900D4200511831628
:1004A000051178308312B900D42005158316051183
:1004B0005A308312B900D420051583160511C830AF
:1004C0008312B900D42005118316051178308312E8
:1004D000B900D42005158316051102308312B80027
:1004E000C830B900D420B80B702A05118316051145
:1004F0000A308312B900D420051583160511643023
:100500008312B900D4200511831605118312360811
:10051000703C031DC72A3708173C031DC72A051561
:1005200083160511C8308312B900D4200511831633
:10053000051178308312B900D420051583160511F2
:1005400002308312B800C830B900D420B80BA32AF7
:1005500005158316051164308312B900D4200511E6
:100560008316051178308312B900D420051583163F
:10057000051102308312B8009630B900D420B80BB0
:10058000BC2A0511831605118312B701B601831623
:0405900034296300A7
:02400E00F43488
:00000001FF
